:100000000EC01BC01BC019C018C02AC016C015C026
:1000100014C013C012C011C010C00FC00EC01124F4
:100020001FBECFEDCDBF10E0A0E6B0E001C01D9235
:10003000A136B107E1F78FD0BDC0E2CF1F920F927A
:100040000FB60F9211248F93809160008F5F809381
:10005000600012BE8F910F900FBE0F901F901895E9
:100060001F920F920FB60F9211240F931F932F938D
:100070003F934F935F936F937F938F939F93AF9330
:10008000BF93EF93FF9380916000803118F184E07B
:1000900088BB30E0A0EBB4E060E87EE304E114E06C
:1000A00040E951E015C008BBCD010197F1F718BB3D
:1000B000CB010197F1F72F5F2A30A9F784EF91E088
:1000C000FA013197F1F70197D9F73F5F343169F1C0
:1000D00020E0E9CF80916000803140F580916000A0
:1000E0008B3020F184E088BB30E0A0EBB4E060E826
:1000F0007EE304E114E040E951E015C008BBCD0106
:100100000197F1F718BBCB010197F1F72F5F2A3068
:10011000A9F784EF91E0FA013197F1F70197D9F748
:100120003F5F323011F020E0E9CF18BA1092600042
:10013000FF91EF91BF91AF919F918F917F916F91BF
:100140005F914F913F912F911F910F910F900FBE93
:100150000F901F90189588E181BD11BC18BA84E1F9
:1001600087BB1ABC83E083BF82E089BF80E28BBF7C
:1001700088E085BB88EE93E020E931E0F901319712
:10018000F1F70197D9F720E034E060E47CE940E939
:1001900051E038BBCB010197F1F718BA88EE93E034
:1001A000FA013197F1F70197D9F72F5F2A3089F7D4
:0801B0007894FFCFF894FFCF13
:00000001FF
